:100000002CC0C3C143C042C041C040C03FC03EC07D
:100010003DC03CC03BC03AC039C038C037C036C014
:1000200035C034C033C00403090448032F651203EC
:1000300054521203303112011001FF000008C016A3
:10004000DC05000101020301090212000101004068
:100050003209040000000000000011241FBECFED93
:10006000CDBF10E0A0E6B0E0ECE2F6E002C0059003
:100070000D92A236B107D9F710E0A2E6B0E001C0B8
:100080001D92A639B107E1F745D0CEC2B9CFFC0128
:100090009181892F807382BB292F2F70E1F482E632
:1000A00090E090937B0080937A0089E480936200D3
:1000B00083E48093630083E58093640082E380930C
:1000C000650080E3809366008093670089E38093F6
:1000D000680087E0089589E690E090937B00809324
:1000E0007A00213019F4828187BB0FC0223019F4C5
:1000F000828188BB0AC0233021F486B380936900D3
:1001000002C0263011F481E0089580E0273009F420
:1001100081E008958FEF87BB85E588BB8BEF81BBBE
:1001200080E282BB83EF81BB8B9A20E040E157E203
:1001300004C0A895CA010197F1F72150D1F78B9817
:1001400085E083BF0AD07894A8950ED008B601FE4A
:10015000FBCF88B7826088BFF7CF85B7836085BF44
:100160008BB780648BBF08950F931F93CF93DF935A
:1001700090917C0019160CF093C020917900809129
:1001800078008D3209F082C08AE5809361009B304F
:1001900009F07CC0CCE0D0E0C21BD109C058DF4FD1
:1001A0009881892F807609F063C01092750089814B
:1001B000882381F49F7119F481E080937500109277
:1001C000760085E790E090937B0080937A0090E83A
:1001D00022E055C0853021F48A8180937D003DC0A6
:1001E000863071F58B81813019F486E390E004C08C
:1001F000823049F488E490E090937B0080937A0009
:1002000090EC22E13CC08330C1F58A81882319F447
:1002100086E290E00EC0813019F48AE290E009C0D5
:10022000823019F48EE290E004C0833031F582E32D
:1002300090E090937B0080937A0090EC24E01FC0C4
:10024000883019F48FE790E00CC0893021F48A815E
:1002500080937F0002C08A3011F090E80FC085E7DC
:1002600090E090937B0080937A0090E821E007C0B3
:10027000CE010DDF282F90E802C090EC20E08F81A6
:10028000882339F48E81821728F003C090E880E03B
:1002900001C0822F90936B008093600010927C00CD
:1002A0008091610084FF49C0809160008F3F09F414
:1002B00044C0182F893008F018E0811B809360003B
:1002C00080916B0080FD02C00BE401C003EC8F5FE6
:1002D00080936B0020917A0030917B0086FD05C0F1
:1002E000D901912FEDE6F0E011C0ADE6B0E080E07D
:1002F00090E006C0F901E80FF91FE491ED93019633
:100300001817C1F705C08D91819391509923D9F7A2
:10031000F901E10FF11DF0937B00E0937A00612F6A
:100320008DE690E02ED0183019F08FEF80936000AA
:1003300000936C001C5F109361009AE080B38C7096
:1003400031F49150D9F710927D0010927700DF912F
:10035000CF911F910F910895A82FB92F80E090E0C1
:1003600041E050EA60956F5F58F42D9138EF822795
:100370009795879510F0842795273F5FC8F3F3CFB3
:100380000895EADF8D939D930895CF93CFB7CF93D0
:10039000839BFECF839B09C0839B07C0839B05C0C3
:1003A000839B03C0839B01C0A1C0DF93C0917900F0
:1003B000DD27C058DF4F839B02C0DF91EBCF2F9327
:1003C0000F931F9300B32FEF03FB20F94F933F933D
:1003D00010B34FEF012703FB21F93BE031C04E7F03
:1003E000012F10B3216028C0102F4D7F2260000024
:1003F00000B329C04B7F2460012F000010B32BC035
:1004000010B3477F28602AC04F7E00B320612CC004
:100410004F7D10B320622FC04F7B00B3206432C0E9
:10042000422700B349934FEF0000102713FB20F938
:1004300010B31C70C9F1297F91F2012703FB21F948
:1004400000B3237F89F2315058F1102713FB22F9B2
:1004500010B3277E79F2012703FB23F92F7C81F269
:1004600000B3102713FB24F92F7971F200C010B3E9
:10047000012703FB25F92F7359F200C000B31027A1
:1004800013FB26F9223040F200C010B3012703FB12
:1004900027F9243028F64F77206810B30000F9CFF1
:1004A00010E41ABF002717C03B503195C31BD04042
:1004B00010E41ABF0881033CE9F00B34D9F0209115
:1004C00077001981110F1213EDCF093641F10D326A
:1004D00011F0013E39F700937E003F914F911F913B
:1004E0000F912F91DF91CAB7C6FD52CFCF91CFBFE9
:1004F000CF91189500917E00002379F310917C0034
:10050000112349F534304AF130937C000093780090
:10051000109179003BE0311B309379001EC00091AF
:100520007C000130C4F40AE53091610034FD17C04D
:1005300000936100CCE6D0E016C0052710E002BBB6
:100540001FC0052722C0052727C005272CC0052767
:1005500010E002BB33C04AE503C042ED01C0432FA7
:10056000C4E1D0E032E011B31C60939A02B311BB36
:100570005F935CE020E820FF052702BB27951795D5
:100580001C3FD8F620FF0527279502BB17951C3F77
:10059000C0F620FF05272795179502BB1C3F98F64C
:1005A00020FF0527279517951C3F02BB70F600C05A
:1005B000499120FF052702BB279517951C3F38F668
:1005C00020FF0527279502BB17951C3F38F520FF14
:1005D00005272795179502BB1C3F10F520FF05271F
:1005E000279517951C3F02BBE8F4242F3A9519F67E
:1005F000037F5F9102BB10917D00110FC651D04067
:1006000011F01093770010E41ABF086011B3137F44
:10061000402F437F02BB11BB42BB5FCF0527D3CF27
:0C0620000527D8CF0527DDCFF894FFCFC9
:02062C00FF5A73
:00000001FF
